:020000040000FA
:1000000083160313810100298B138B1B0428AD0079
:10001000030EAE0083010A08AF008A0183130408AF
:10002000B0008B1838280B182A288C1A21280C1895
:100030001A289428C103031D1F28291529100C1004
:1000400094281A08AA002714831603138C1283120B
:1000500003138E28861F90288B115030B100B10BEE
:100060002F281F151F1932281E08BD00A817902819
:10007000281C5E283208073C031C4428331C051248
:1000800033180516B30C92283208083C031C4D287F
:10009000A81C0512A818051692283208093C031C52
:1000A0005728831603130516831203139228320868
:1000B0000B3C031C9228B20128109328B208031DA0
:1000C0006428051A892892283208083C031C7028E5
:1000D000051EB313051AB31703199228B30C9228FF
:1000E0003208093C031C75289228051E8A28281905
:1000F0008228A71783160313061083120313061012
:100100000B128C2836083302031D8B282811B201EC
:1001100093288B288B28B301B20193288C12942842
:100120000B109428B20A8B10300884002F088A0024
:100130002E0E8300AD0E2D0E09003308B400F03CE6
:10014000031DA528A714A711232BA71C992AA710C4
:100150003308123C0319AF283308593C03192711FF
:100160003308583C031DD428271EC5282712ED301C
:10017000B300CF24B624FA30DC2435113508B3009F
:10018000CF24B624FA30DC24232B2716ED30B3001D
:10019000CF24B624FA30DC2435153508B300CF243B
:1001A000B624FA30DC24232B3308113C031DDA2853
:1001B000A712642B3308143C031D232B27139B2BFE
:1002000002309F0083120313091083160313091091
:1002100083120313831603130614051601138312A6
:1002200003138B100B168316031305148617831202
:100230000313C1309F000B108B15F8308B058C0118
:100240008D018B170230B500B201A701A801A901E9
:1002500083160313013088058312031388120813D1
:100260008813E130880504303724033047246124A3
:10027000013037240830472461240130372402300C
:10028000472461240130372428304E240C304E247A
:1002900001304E24083037242830B700B80126300A
:1002A000A50006308A002508263C00265024A50B10
:1002B0005129FF30B300CF24B624ED30B300CF2452
:1002C000B624FA30DC243508B300CF24B624FA3043
:1002D000DC24ED30B300CF24B624FA30DC2435140E
:1002E0003508B300CF24B624FA30DC24FF30A00058
:1002F0000430852480303724F030A0000430852479
:10030000C0304E242830A50006308A002508283C3D
:100310004F265024A50B842929141730BE00033022
:10032000BF0055309C24A81B1F25A71B9D20291802
:100330009329AA2480303724F030A000043085248B
:1003400080303724F030A000043085248B133E0821
:100350008316031399001811831203139817831639
:1003600003138C169816831203130B171816F83004
:100370008B058C018D018B1701304E242730A50091
:1003800006308A002508273C2726A600B224260826
:100390005024A50BC0290D30B2240A30B2240A30F3
:1003A000B224A71B9D202718E624A81B1F25D129AE
:1004400082070034393400343534333431343234B3
:1004500032340034303438343634343409347E3471
:10046000003400342D2B2B2B00342F2B71343134DE
:100470000034003400347A347334613477343234E5
:1004800000340034633478346434653434343334C1
:1004900000340034203476346634743472343534A5
:1004A000003400346E34623468346734793436345E
:1004B0000034003400346D346A34753437343834E1
:1004C000003400342C346B3469346F3430343934B4
:1004D000003400342E343F346C343B3470342D34CB
:1004E000003400340034273400345B342B340034BF
:1004F000003400342B2B1A2B5D3400347C34003450
:10050000003400343C3430342E3432343534363414
:1005100038340034003431342B3433342D342A341D
:10052000393400340834003400343134373434344E
:100530003734A71DAB2AA71AAB2A271BAB2A3308CF
:100540004A3C031DA62A2F30B300DF2A33085A3C49
:100550000318AB2A232B3308613C0318C12A0E3041
:10056000B3023308613C031CB82A1930B307C12A0F
:100570003308773C0318C12A3308D23C0319A71566
:10058000232B02308A0033082022B300B30803195A
:10059000232BA71A472B271B352B3308603C031846
:1005A000B42B33087A3C031CB42B3308271ADB2AFC
:1005B000271DDF2ADD2A2719DF2AE03EB30029188C
:1005C000042B3308B2243308083C031DF52A3808ED
:1005D0000319232BB8033808403E8038A5004E2469
:1005E0002030502425084E24232B3308093C031DBA
:1005F000022B3808263C031C002B20305024B80A5C
:100600002030B3007225232B3308613C031D0E2BD1
:100610005125F030A00004308524172B3308733C9B
:10062000031D172B2910F030A0000430852455300D
:10063000C100232B29180034A81680250D30B224C0
:100640000A30B224003483160313061483120313F2
:10065000A7130B16080027150034A716302B2717F1
:10066000B901BA01BB01BC0100343308403C031896
:10067000472B3308463C031C3F2BB3164F2B330844
:10068000603C0318472B3308663C03184F2B330894
:10069000293C0318232B3308393C031C232BB908AE
:1006A000031D562BB90A3308BA00232B390B5C2BD8
:1006B000B90A3308BB00232B3908023C031D232B46
:1006C000B90A3308BC00232BB9080319232B303097
:1006D000BA02BB02BC02B903031D712B3A08B30076
:1006E0008B2BB903031D7B2B03308A003A088D2323
:1006F0003B07B3008B2B3A08023C031C232B03302F
:100700008A003A080A3E8D23BA003B088D23BA07B7
:100710003C083A07B300B901DF2A820700340A34E3
:1007200014341E34283432343C34463450345A3471
:1007300000346434C834B9080319232B3030BA02AA
:10074000BB02BA1EA52B2730BA02BB1EA92B27302D
:10075000BB02B903031DAF2B3A08B300B22B3A0E0C
:100760003B04B300B901DF2A271DDF2A33080D3C03
:100770000318DF2A3408613C031CDF2A34083C3CA0
:100780000318C52B3D30B402CE2B3408243C03188B
:10079000CC2B2330B402CE2B0430B40703308A00B4
:1007A0003408D423B300DF2A820726342A342434C1
:1007B00023343C34003400340034293428340034E9
:1007C00025343E342F3400343A3400345F346034FE
:1007D0005E340034223400347B343D340034213420
:1007E0000034003400347D3400345C340034403450
:0407F00000343E345F
:10086000A000810183160313C03081050800A00099
:10087000810183160313C030810501308104831286
:1008800003130B110B1D422CA00B412C0800A200DE
:10089000E1308805220D1E39880408002816512CE5
:1008A0002812A3006A24281E88172308230E472431
:1008B0006124230847246124E13088058813081344
:1008C000080088160000881208001830A200A20B49
:1008D000672C08008813A815831603131E3088049C
:1008E000831203130817000088166524081EA81138
:1008F000881265246124A819742C08138316031325
:10090000E1308805831203130800A10081018316DA
:10091000031307308100831203130B11091497246A
:10092000091097240B1D8E2CA10B8D2C080020087C
:10093000A200A20B992C0800C10029118E018F0181
:100940000C10831603130C14831203130B1731308E
:1009500090000800831603130C1083120313101069
:10096000291108000C1EB22C990008000B128316E6
:10097000031306100512831203130610051220300C
:10098000A000A00BC12CB20183160313061483121E
:10099000031328148B100B162818CC2C0800A20067
:1009A0000830A300A4012218A40AA20CA30BD32C84
:1009B000A810241CA8140800B60028152919E32C37
:1009C0002819DE2C08002811B20108002A08AC0002
:1009D000FA24A91CF42C2B08AC00FA24A910981CAA
:1009E000F42C181218111816831603138C16831280
:1009F000031308002C08083C031D082D37080319B1
:100A00001D2DB703370880384E24203050241D2D6B
:100A10003708273C03180E2DA81280253708803888
:100A20004E242C080D3C031C1A2D031D1D2DA8124D
:100A300080251D2D2C085024B70A27100800F030FF
:100A4000A000043085240B30A50006308A0025085C
:100A5000A226FD3EA6003D02031C332D26083D02C2
:100A6000063C0318352DA50B252D06308A002508D8
:100A7000AF262918412DB224B3007225A8138B1577
:100A80000800A5002A3C031D472D51254C2D2508A3
:100A9000233C031D4C2D2910A8135530C1008B1584
:100AA0000800C001BF0A3F08073C0318582DBF01CA
:100AB0003F08A6000319602D0430C007A60B5C2D6B
:100AC000C6304E240430A60006308A00400878263E
:100AD0005024C00AA60B642D06308A003F089926D0
:100AE000BE0008003808273C0318782DA81680257A
:100AF0003808403E80384E2433085024B80A080095
:100B00002830A81A8E2DB70080304E242030502473
:100B1000B70B862D80304E24B7010800B800C030D6
:100B20004E2420305024B80B912DC0304E24B801F3
:020B30000800BB
:100C0000820743347534733474346F346D3469340B
:100C10007A346134743469346F346E3420346F3410
:100C200066342034533465347234693461346C343E
:100C3000203443346F346D346D3475346E3469341C
:100C400063346134743469346F346E343A348207F7
:100C500050344934433431343634463437343734FD
:100C600020344134543420344B3465347934623484
:100C70006F34613472346434203442346F347834E5
:100C80002034563432342E343034353420347334F6
:100C9000743461346E3464342D34623479348207B0
:100CA0005234533432343334323420342034203408
:100CB000393436343034303420346234613475346D
:100CC00064342034203461342F342A3420346134A5
:100CD0006C347434653472342034203473342F34DB
:100CE00023342034733465346C34653463347434A1
:100CF00082072034203431343234203420343234EA
:100D000034342034203434343834203420343934EA
:100D100036342034313439343234203433343834B6
:100D20003434203435343734363431343134353496
:100D300032348207BF345F342F3417340B34053418
:100D40000334013482074E345E346C347C348B348B
:100D50009B34AC34BE34CF34E134F334FF348207F7
:100D60002A3437343434313430343834353432344E
:080D70002334393436343334E6
:02400E00F23F7F
:00000001FF
